:0600000000308A00142804
:10000800A00003088301B20083120C1C0E2885127D
:1000180010100C10831232088300A00E200E090065
:10002800213084002C3020208316FF239000830188
:080038005A2804068001840A25
:100040000406031D1D286400003483121F119F1431
:100050009F1828281E08AA00AB01AB00AA0183162E
:100060001E088312AA070318AB0A0A30AE00AF01BC
:100070002B08AD002A08AC0015213008A400310877
:10008000A5001E30AE00AF012B08AD002A08AC0061
:1000900015213008A6003108A7000C30AE00AF01D2
:1000A0002B08AD002A08AC0015213008A800310843
:1000B000A9000800000032308312AA00AB018312AD
:1000C000FE20051185121B308316850061309F00CC
:1000D000813083129F00073099001F143030900048
:1000E0006430AA00AB01FE2083160C140B178B178B
:1000F0008312851DB22021188620051E8620A11896
:10010000B2202520DE202110A110782883121010A3
:1001100023088F0022088E00FF308500AA01AB0162
:10012000972885199428A114AA0A0319AB0A27084D
:100130002B02031D9D2826082A02031C9128051165
:10014000AA01AB0129082B02031DA82828082A02AE
:100150000318B028851DA114AA0A0319AB0AA22806
:10016000101408008312101023088F0022088E003C
:10017000FF308500AA01AB01C328051AC02821144D
:10018000AA0A0319AB0A25082B02031DC928240853
:100190002A02031CBD280511AA01AB0129082B0264
:1001A000031DD42828082A020318DC28051E211460
:1001B000AA0A0319AB0ACE281014080083121F15CF
:1001C0009F149F18E1281E08AA00AB01AB00AA01EA
:1001D00083161E088312AA070318AB0A2B08AD006A
:1001E0002A08AC000630AE000310AC0DAD0DAE0B0E
:1001F000F4282C08A2002D08A30008000A30AE0045
:10020000AF0183122A08AC002B08AD00152130087D
:10021000AA003108AB001029AA080319AB03AA03EE
:100220002B082A04031908000C29B001B10103109E
:10023000AF0CAE0C031C23292C08B0072D080318A3
:100240002D0AB1070310AC0DAD0D2E082F040319B4
:040250000034172936
:02400E00C43FAD
:1042000065007500010063006300400074007500E4
:1042100074002E0062007900000000000000000021
:00000001FF
